:100000001DC02AC029C028C027C026C025C024C0C2
:1000100023C022C0798D9AA2AAFFA1A3A3A3A3A360
:10002000A1A1A1A1A103146EFFFFFF000000000029
:10003000000000073889FFFCFEFDFF0011241FBEF1
:10004000CFE9CDBF10E0A0E6B0E001C01D92A3361D
:10005000B107E1F76AD033C1D3CF26EB33E003C059
:10006000F9013197F1F70197D8F7089588EE93E0F9
:10007000F4CFCF93C09162008C2F8F5F8F738093EA
:1000800062006091600090E00CD16FEF8C2F90E0E7
:10009000CF9107C1CF931092620008C08C2F90E0DF
:1000A000F8D08F3F41F4CF5FC0936200C0916200EF
:1000B000C034A0F302C080936000CF9108958111F5
:1000C00004C0611102C091EA9FBD89BD66BF089559
:1000D00090E0FC01E65EFF4FE491EFBDFC01EB5DBB
:1000E000FF4F6491FC01E05DFF4F8491E8CF369AA9
:1000F0003699FECF85B108951F93CF93DF93C82F14
:1001000014E1D1EA0CC019BC16BF84E690E0A5DF6B
:10011000DFBD19BC16BE80E991E09FDFC150C1115F
:10012000F2CFDF91CF911F910895A39A83E687B90B
:1001300086EC86B93699FECF369A3699FECFC5B190
:1001400080E188BBB99AB89A81EA8FBD81E083BF0C
:10015000A1DFC63F40F0809160008F5F8093600018
:100160008730B0F013C0C53B68F0809160008730E5
:1001700009F40CC0882311F0815001C08AE08093FB
:10018000600006C080916100811102C01092600081
:1001900070DFBB9AC39AA29A81E687B986EC86B9CA
:1001A000369AC0E010E00FEF81EAF82E95E0E92ED4
:1001B00080916000E82FF0E0E05DFF4FD491DD3FDB
:1001C00059F409BD16BE82E390E047DFFFBC19BCBD
:1001D00016BE82E390E031C0DC3F81F4D4E009BD7B
:1001E00016BE85E090E039DF19BC06BF81E490E0DF
:1001F00034DFD150A1F780ED92E01FC0DE3F81F4E3
:1002000076DF982F80E001C08F5FE82FF0E0EC5E92
:10021000FF4FE491E917C0F36FDF28DF27DF0EC03F
:1002200057DF1F5F1B3538F0DF3F29F4E092600095
:1002300085E04EDF1EDF84EF91E00FDF349BB8CF07
:1002400085B1813718F5CF5FC83008F1C0916000E3
:10025000C73098F4CC2311F0C15010C0FFBC19BCBA
:1002600016BE85B7877E806185BF85B7806285BFF2
:10027000889585B78F7D85BF01C0C2E08C2F28DFB0
:10028000C0936000F6DE8AEF90E0E7DEC0E0369AC9
:100290008FCFE199FECF1FBA8EBBE09A99278DB31D
:1002A0000895262FE199FECF1CBA1FBA8EBB2DBB35
:1002B0000FB6F894E29AE19A0FBE01960895F89469
:0202C000FFCF6E
:00000001FF
